:100000000C9476000C94EA010C9493000C949300E9
:100010000C9493000C9493000C9493000C94930014
:100020000C9493000C9493000C9493000C94930004
:100030000C9493000C9493000C9493000C949300F4
:100040000C9493000C9493000C9493000C949300E4
:100050000C9493000C9493000C9493000C949300D4
:100060000C9493000C9493001A034A0061006700FB
:100070007500610072002000410074006100720090
:100080006900180372006100700068006E0065006E
:1000900074002E006E0065007400040309040A0356
:1000A000310030003000300005010905A1010901CF
:1000B000A10009300931150026FF0075089502815D
:1000C00002C00509190129111500250175019511B5
:1000D0008102750195078103C01201010100000032
:1000E000089B2818000201010203010011241FBE11
:1000F000CFEFD4E0DEBFCDBF11E0A0E0B1E0EEEB8A
:10010000FAE002C005900D92A833B107D9F721E0BB
:10011000A8E3B1E001C01D92A838B207E1F70E9440
:10012000A7040C945D050C940000CF93C62F20917A
:100130005D0124FF07C020915E0138E8232720934A
:100140005E0103C02AE520935D01DC01EFE5F1E0EB
:100150009C2F9E0F8D918193892F8E1B1816D4F39F
:100160006C2F8FE591E00E94E601CC5FC0935D01AA
:10017000CF910895CF93DF9380916E01835087FDD7
:10018000ABC090916B0120916A012D3209F0A2C0A1
:10019000883009F09FC0CCE0D0E0C91BD109CE580F
:1001A000DE4F83EC809352018AE580930101109227
:1001B00038018881807621F0CE010E94520381C0EF
:1001C0009A8110925B018981811106C010925C01B5
:1001D0002BE531E082E071C0853019F490936F0116
:1001E00069C0863009F050C08B81813009F442C06B
:1001F000823029F4CE010E94240390E042C0833073
:1002000061F5911109C08AE990E090936D018093A6
:100210006C0190E484E035C0913049F482E890E0CC
:1002200090936D0180936C0190E488E12AC0923034
:1002300049F488E690E090936D0180936C0190E41E
:100240008AE11FC09330D9F48EE990E090936D015C
:1002500080936C0190E48CE014C0813249F48BE40B
:1002600091E090936D0180936C0190E489E009C066
:10027000823229F4CE010E94240390E402C090E46B
:1002800080E0909338011DC0883069F0893019F4FE
:10029000909371010FC08A3049F08B3059F48BE490
:1002A00080935E0107C021E731E002C02BE531E019
:1002B00081E003C02BE531E080E030936D012093B5
:1002C0006C019F81911104C09E81981708F4892FB9
:1002D0008093000110926E018091010184FF47C05C
:1002E000809100018F3F09F442C0C82F893008F087
:1002F000C8E08C1B809300018091520198E8892707
:1003000080935201CC2331F120916C0130916D0129
:100310008091380186FF0BC0A3E5B1E0F9018C2F75
:100320008A0F94919D9331968A13FBCF09C0D9010E
:10033000E3E5F1E08C2F8E0F9D9191938E13FCCF0E
:100340008FEF8C0F90E00196820F931F90936D01B9
:1003500080936C016C2F83E591E00E94E601CC5FF5
:10036000CC3019F08FEF80930001C093010184E13C
:1003700099B1957031F48150D9F710926F011092B4
:100380006901DF91CF910895E9E6F0E08081826014
:100390008083E89A8BE480935E018AE580935D0117
:1003A0000895A82FB92F80E090E041E050EA6095D1
:1003B00030E009C02D9182279795879510F084270A
:1003C0009527305EC8F36F5FA8F30895EADF8D9339
:1003D0009D930895CF93CFB7CF93C395489BE9F7EB
:1003E000489B09C0489B07C0489B05C0489B03C069
:1003F000489B01C0A3C0DF93C0916B01DD27CE589D
:10040000DE4F489B02C0DF91EBCF2F930F931F93DA
:1004100009B12FEF00FB20F94F933F9319B14FEF34
:10042000012700FB21F93BE031C04E7F012F19B1BC
:10043000216028C0102F4D7F2260000009B129C023
:100440004B7F2460012F000019B12BC019B1477FE9
:1004500028602AC04F7E09B120612CC04F7D19B1A0
:1004600020622FC04F7B09B1206432C0422709B1FE
:1004700049934FEF0000102710FB20F919B11570B8
:10048000C9F1297F91F2012700FB21F909B1237FEE
:1004900089F2315058F1102710FB22F919B1277E4B
:1004A00079F2012700FB23F92F7C81F209B1102793
:1004B00010FB24F92F7971F200C019B1012700FB5C
:1004C00025F92F7359F200C009B1102710FB26F946
:1004D000223040F200C019B1012700FB27F9243077
:1004E00028F64F77206819B10000F9CF11E01CBB46
:1004F000002719C03B503195C31BD04011E01CBBF5
:100500000881033CF9F00B34E9F02091690119816D
:10051000110F1213EDCF4A81441F093641F10D32FC
:1005200011F0013E29F7009370013F914F911F9107
:100530000F912F91DF91CCB3C0FD4FCFCF91CFBFA3
:10054000CF91189520917001222379F310916E01BB
:10055000112369F534306AF130936E0120936A01FA
:1005600010916B013BE0311B30936B0122C0009175
:100570006E010130E4F40AE54F7049F43091010155
:1005800034FD19C000930101C2E5D1E018C03091DB
:100590005D0134FD10C000935D01CEE5D1E00FC0D8
:1005A0002795A8F45150A9F4220F0000F9CF4AE58D
:1005B00003C042ED01C0432FC4E1D0E032E01AB1E4
:1005C0001560589A1AB90BB120E415E05F93012722
:1005D00056E00BB9279520F4515021F4220FF9CFA2
:1005E000012756E000003B5A0BB9D0F2279528F4BA
:1005F000515029F4220F0000F9CF012756E027952A
:100600000BB920F4515021F4220FF9CF012756E005
:10061000299133230BB921F60A7F10916F01110F35
:10062000C651D0400BB911F01093690111E01CBB09
:1006300001601AB11A7F402F4A7F5F9100C000C04D
:100640000BB91AB94BB971CFFC018081807641F5A5
:100650009181963031F593819230D1F0923269F0E8
:100660009130F9F4809143019091440190936D0190
:1006700080936C0180914201089580914601909190
:10068000470190936D0180936C018091450108951D
:1006900082E091E090936D0180936C0182E2089575
:1006A00080E008952AE331E030936D0120936C01DE
:1006B000FC0120812076203299F48181813081F4FF
:1006C000E0914001F09141010088F189E02D8AE339
:1006D00091E00995E0914001F091410180810895F8
:1006E00080E00895009741F025E0EDE4F1E0DC01C1
:1006F00001900D922A95E1F785E0EDE4F1E0A8E4A0
:10070000B1E001900D928A95E1F70895EF92FF9282
:100710001F93CF93DF93CDB7DEB767970FB6F894EB
:10072000DEBF0FBECDBF80E88A8389831B821C8217
:100730001D821E821F827E0188E0E80EF11C8CE083
:10074000D7011D928A95E9F7FE01749680E090E04A
:1007500040E250E09A01082E02C0359527950A9490
:10076000E2F768B1122F1095612368B967B1622B67
:1007700067B9AFE6B7E11197F1F700C0000076B1B5
:100780007370708363B168736695672B6083189B81
:1007900002C06062608337B1312337B938B1322B80
:1007A00038B90196319684309105A1F69F8981E090
:1007B00091FB662760F968276F835C89752F7170DC
:1007C00078277E834D89E42FE170E827ED833E8909
:1007D000F32FF170F827FC83292F217028272B8312
:1007E00054FB112710F918271A8744FB112710F919
:1007F0001827198734FB112710F91827188794FD3B
:1008000002C08FEF898311E053FB882780F981278D
:100810008D8743FB882780F981278C8733FB8827C6
:1008200080F981278B8793FF198211E052FB88277B
:1008300080F98127888B42FB882780F981278F8761
:1008400032FB882780F981278E8792FD02C08FEFC7
:100850008A8381E055FB552750F958275B8B45FB70
:10086000442740F948274A8B35FB332730F938278E
:10087000398B95FF1A82F1112260E1112460711108
:10088000286061112061F70180E090E030E2419141
:100890004111232B0196330F83309105C1F780E07E
:1008A00090E041E030E0E4E0F0E0EC0FFD1FE80F05
:1008B000F91F67816111342B440F0196883091052F
:1008C00091F7898180934D018A8180934E01209315
:1008D0004F01309350015093510167960FB6F89431
:1008E000DEBF0FBECDBFDF91CF911F91FF90EF9084
:1008F0000895CF93CFB7F89417B88FEF88B914B88D
:1009000085B90E948603CFBFCF91089580912401BD
:1009100090912501892B31F010922501109224012C
:1009200081E0089545E050E068E471E08DE491E0F5
:100930000E945005089588EA90E090932B018093DF
:100940002A0186E291E0089582E190E0089581E035
:1009500084B98EEF85B917B88FEF88B988EF8BB956
:1009600085E08AB914BC85BD82E08093B00087E041
:100970008093B10082E38093B3000E949B04FC014A
:100980009093410180934001848195819093470128
:1009900080934601828180934501808591850097EF
:1009A00031F09093440180934301868108C089ED22
:1009B00090E090934401809343010E94A4048093AB
:1009C00042018091450180931B012FE088E190E076
:1009D0000FB6F894A895809360000FBE2093600036
:1009E000E0914001F09141010284F385E02D0995E9
:1009F0000E94C4018BB18A7F8BB98AB185608AB9A4
:100A000087EC9FEA0197F1F700C000008AB18A7F66
:100A10008AB9789411E0D0E0C2E0A8950E94BA00AB
:100A2000112341F0E0914001F09141010484F585EA
:100A3000E02D0995B99B16C0C7BBD11115C0E09137
:100A40004001F09141010484F585E02D0995E09184
:100A50004001F09141010684F785E02D099581114F
:100A600003C01CC0DD23D1F080915D0184FD03C073
:100A7000D1E010E0D2CFE0914001F0914101008837
:100A8000F189E02D8AE391E00995E0914001F09130
:100A9000410160818AE391E00E949500D0E0E9CFB6
:100AA000FB01DC0104C08D910190801921F44150BB
:0E0AB0005040C8F7881B990B0895F894FFCFAB
:100ABE00FF5A090222000101000032090400000160
:100ACE000300000009210101000122000007058139
:100ADE000308000A010005003100000000000000BC
:080AEE007904860386047203FB
:00000001FF
